:020000002D28A9
:080008009400030895007F300D
:1000100081000B110D08031D17280F08031D05157E
:100020001008031D85141108031D051423280F084B
:100030000D020319051110080D020319851011088E
:100040000D02031905108D0A0D08203C03198D01BE
:1000500015088300940E140E0900003085008316E5
:10006000D030810018308500FF30860083122030A8
:1000700092008D01602160206B20772082208E20ED
:1000800099207720822060206B20772082208E208C
:100090009920772082206020A520B220CC20D92072
:1000A000A520B220CC20D9206B20602077208E2084
:1000B000F320E620F320642101210E212721372897
:1000C00012089A008F019001910149219A030319A6
:1000D00008008F0A652812089A001F308F009001CF
:1000E000910149219A03031908008F03712812080E
:1000F0009A008F019001910149219A030319080088
:10010000900A7C2812089A008F011F3090009101FC
:1001100049219A03031908009003882812089A00BD
:100120008F019001910149219A0303190800910A56
:10013000932812089A008F0190011F3091004921E5
:100140009A030319080091039F2812089A001F3090
:100150008F009001910149219A0303190800900A28
:100160008F03AB2812089A008F011F309000910175
:1001700049219A0303190800910A9003B82812082C
:100180009A008F0190011F30910049219A030319B1
:1001900008008F0A9103C52812089A008F01900168
:1001A0001F30910049219A0303190800900A910316
:1001B000D22812089A008F011F3090009101492126
:1001C0009A03031908008F0A9003DF2812089A0087
:1001D0008F019001910149219A03031908008F0AA8
:1001E000900A910AEB2812089A001F308F009000A5
:1001F000910049219A03031908008F03900391038A
:10020000F928051540210511851440218510051494
:100210004021051085144021851008000515432153
:1002200005118514432185100514432105108514FB
:10023000432185100515432105118514432185109F
:100240000514432105108514432185100800051568
:10025000432185144321051443213C2143213821A6
:1002600043213C214321382143213C2143210800E3
:1002700005158514051408000511851005100800E2
:100280000A3099004E29053099004E290130990015
:100290004E29303098006630970059297B309800FD
:1002A000DD309700970B5229980B5029990B4E2956
:1002B0000800970B592918080319080098035929B1
:1002C0008101A0308B0008008B138B1B64298B01EC
:0202D000080024
:02400E00F93F78
:00000001FF
